:100000008316FF30853000308600C13081008312B6
:1000100003018501860191018D019201FF308C0061
:10002000930094009500E7308100051E012B010824
:10003000031D1728E73081008D0A03198C0A14303C
:100040000C020319002885192D281408031D3528D2
:10005000FF309400061693014E2814080319352822
:10006000061294011728950317281208031D472824
:100070001508031D33281308031D172806148615B9
:100080000611FF309200930001308E0017288E0B6E
:100090001728061086110615920117280C08031D53
:1000A0005A280D08263A0319862826300D02031C0B
:1000B00086286B280C08013A0319632801300C02CA
:1000C000031882286B280D08903A03198228903073
:1000D0000D020318822825308D02031C8C030310A7
:1000E0008C0C8D0C03108C0C8D0C743091000D0851
:1000F00011020A108A1400228F008C018D010F0852
:100100009500172800308F0086107D288F018614F7
:020110007D2848
:1004000082070034013401340234033403340434E9
:100410000434053405340534053406340634073411
:1004200007340834083409340A340B340B340C34E0
:100430000C340D340D340E340E340F340F341034AC
:10044000103411341134123412341334133413347D
:10045000143414341534153416341734183418344D
:10046000193419341A341A341A341B341B341C341A
:100470001C341D341D341D341D341E341E341E34F2
:100480001F341F34203420342134213421342234C9
:10049000223423342334243424342534253425349D
:1004A0002634263427342734283428342834283472
:1004B000293429342A342A342A342B342B342C344A
:1004C0002C342D342D342D342E342E342F342F341F
:1004D00030343034303431343134323432343234F4
:0E04E00032343234323432343234323408346E
:10060000002886140612851D062B122B0616E730CD
:10061000960004309700960B0E2B970B0B2B102B8C
:100620001E2B012B06165F309600EB309700960BC1
:100630001A2B970B172B1C2B1E2B012B06140611A4
:100640008F30960002309700960B272B970B242BA8
:08065000292B06100615012BF1
:02400E00F93F78
:00000001FF
